:020000040800F2
:1000000000800120692A0008811B0008831B00086A
:10001000851B0008871B0008891B000800000000E2
:100020000000000000000000000000008B1B000822
:100030008D1B0008000000008F1B0008911B0008AA
:10004000B92A0008B92A0008B92A0008B92A000804
:10005000B92A0008B92A0008B92A0008B92A0008F4
:10006000B92A0008B92A0008B92A0008B92A0008E4
:10007000B92A0008B92A0008B92A0008B92A0008D4
:10008000B92A0008B92A0008B92A000800000000AF
:10009000000000000000000000000000B92A000875
:1000A000B92A0008B92A0008B92A0008B92A0008A4
:1000B000B92A0008B92A0008B92A0008B92A000894
:1000C000B92A0008B92A0008B92A0008B92A000884
:1000D000B92A0008B92A0008B92A0008000000005F
:1000E000B92A0008B92A0008B92A0008000000004F
:1000F000000000000000000000000000B92A000815
:1001000000000000B92A0008B92A0008B92A00082E
:1001100000000000000000000000000000000000DF
:10012000B92A0008B92A0008B92A0008B92A000823
:10013000B92A0008000000000000000000000000D4
:10014000000000000000000000000000B92A0008C4
:10015000B92A0008B92A0008B92A0008B92A0008F3
:10016000B92A0008B92A00080000000000000000B9
:10017000000000000000000000000000000000007F
:1001800000000000B92A0008000000000000000084
:04019000B92A000880
:1001C0000348044B834202D0034B03B118477047E6
:1001D0007000002070000020000000000548064963
:1001E0000B1AD90F01EBA301491002D0034B03B145
:1001F00018477047700000207000002000000000C9
:1002000010B5064C237843B9FFF7DAFF044B13B15E
:100210000448AFF300800123237010BD700000205C
:1002200000000000BC2A000808B5044B1BB10449BB
:100230000448AFF30080BDE80840CFE700000000AD
:1002400074000020BC2A0008014B1868704700BFEA
:100250000000002070B50D4E0D4D761BB61006D077
:10026000002455F8043B01349847A642F9D1094EC1
:10027000094D761B02F022FCB61006D0002455F87A
:10028000043B01349847A642F9D170BD442F0008C1
:10029000442F0008482F0008442F0008024B014655
:1002A000186800F059B900BF00000020024B014659
:1002B000186800F0EFB800BF00000020844641EA53
:1002C000000313F003036DD1403A41D351F8043BCE
:1002D00040F8043B51F8043B40F8043B51F8043B20
:1002E00040F8043B51F8043B40F8043B51F8043B10
:1002F00040F8043B51F8043B40F8043B51F8043B00
:1003000040F8043B51F8043B40F8043B51F8043BEF
:1003100040F8043B51F8043B40F8043B51F8043BDF
:1003200040F8043B51F8043B40F8043B51F8043BCF
:1003300040F8043B51F8043B40F8043B51F8043BBF
:1003400040F8043B51F8043B40F8043B403ABDD22E
:10035000303211D351F8043B40F8043B51F8043BD0
:1003600040F8043B51F8043B40F8043B51F8043B8F
:1003700040F8043B103AEDD20C3205D351F8043B5F
:1003800040F8043B043AF9D2043208D0D2071CBF2B
:1003900011F8013B00F8013B01D30B880380604654
:1003A000704700BF082A13D38B078DD010F00303CA
:1003B0008AD0C3F10403D21ADB071CBF11F8013B3A
:1003C00000F8013B80D331F8023B20F8023B7BE789
:1003D000043AD9D3013A11F8013B00F8013BF9D2B4
:1003E0000B7803704B7843708B788370604670474E
:1003F000830730B548D0541E002A3FD0CAB2034606
:1004000001E0013C3AD303F8012B9D07F9D1032CFD
:100410002DD9CDB245EA05250F2C45EA054536D93B
:10042000A4F1100222F00F0C03F1200EE6444FEA73
:10043000121C03F1100242E9045542E90255103240
:100440007245F8D10CF1010214F00C0F03EB02120B
:1004500004F00F0C13D0ACF1040323F003030433B6
:10046000134442F8045B9342FBD10CF003042CB11B
:10047000CAB21C4403F8012B9C42FBD130BD644638
:100480001346002CF4D1F9E703461446BFE71A4699
:10049000A446E0E7002958D030B551F8043C83B0B9
:1004A000002BA1F10404B8BFE418019000F076F924
:1004B000284A0198136833B1A3420DD9216804EB8F
:1004C000010C63452FD06360146003B0BDE8304079
:1004D00000F066B9A34210D81A465B68002BF9D128
:1004E000116802EB010C644519D02FD3636054608E
:1004F00003B0BDE8304000F053B9116802EB010CC5
:10050000A44516D022D8216804EB010C6345EDD137
:100510001D685B682944C4E900135460D5E723686B
:1005200019441160D1E71D685B682944C4E90013D0
:10053000CAE7246821445418A3421160C5D1D3E905
:1005400000432144C2E90013BFE770470C23036056
:10055000BBE700BF8C000020F8B5CD1C25F00305DB
:1005600008350C2D38BF0C25002D064623DBA9428B
:1005700021D8254F00F012F93A6822B3144603E05F
:1005800063682246FBB11C4623685B1BF8D40B2B27
:1005900015D8636894420CBF3B605360304600F04E
:1005A000FFF804F10B00231D20F00700C21A01D050
:1005B0001B1AA350F8BD0C2333600020F8BD236044
:1005C0001C442560EAE77968C9B12946304600F045
:1005D0001DF8431C0CD0C41C24F00304A04205D019
:1005E000211A304600F012F8013001D02560D5E71D
:1005F0000C233046336000F0D3F80020F8BD3046BD
:1006000000F004F87860E0E78C00002038B5074D72
:100610000022044608462A6002F002FA431C00D079
:1006200038BD2B68002BFBD0236038BD9400002020
:100630000CB410B59CB01EAB6FF00044CDE90614AD
:100640000291084953F8042B059102A901930494DF
:1006500000F086F9029B00221A701CB0BDE8104021
:1006600002B070470802FFFF0EB410B59DB06FF0E6
:1006700000411FABCDE906010491094953F8042B51
:100680000290084C0868019302A9059400F068F9EB
:10069000029B00221A701DB0BDE8104003B07047E5
:1006A000000000200802FFFF000000000000000022
:1006B000000000000000000000000000000000003A
:1006C00090F800F06DE9024520F007016FF0000C92
:1006D00010F0070491F820F040F049804FF000043A
:1006E0006FF00700D1E9002391F840F000F1080015
:1006F00082FA4CF2A4FA8CF283FA4CF3A2FA8CF34D
:100700004BBBD1E9022382FA4CF200F10800A4FAB3
:100710008CF283FA4CF3A2FA8CF3E3B9D1E9042307
:1007200082FA4CF200F10800A4FA8CF283FA4CF33E
:10073000A2FA8CF37BB9D1E9062301F1200182FAF8
:100740004CF200F10800A4FA8CF283FA4CF3A2FAFE
:100750008CF3002BC6D0002A04BF04301A4612BA0C
:10076000B2FA82F2FDE8024500EBD2007047D1E90F
:10077000002304F00305C4F100004FEAC50514F09E
:10078000040F91F840F00CFA05F562EA05021CBF6F
:1007900063EA050362464FF00004A9E7704700BF13
:1007A000704700BF2DE9F0478F689F420C461D46F9
:1007B000164638D88246888910F4906F0ED10868A2
:1007C0003D462A46314600F023FCA2682368D21B2E
:1007D0002B44A26023600020BDE8F0874B690969C3
:1007E00003EB4308236808EBD878A3EB01096B1CE3
:1007F0004FEA68084B444345424684BF9846424608
:10080000430513D511465046FFF7A6FE074608B329
:1008100021694A46FFF752FDA38923F4906343F010
:100820008003A38107E008681F46CAE7504600F02E
:100830006BFC074650B107EB0900A8EB09032761E1
:10084000C4F81480A36020602F46BAE7216950469F
:10085000FFF720FE0C23CAF80030A38943F04003C1
:100860004FF0FF30A381B7E72DE9F04F936883B0D5
:100870009146002B6ED017688D6880460C4608683C
:10088000083744E0A38913F4906F2ED0D4E90415FF
:10089000A0EB010A05EB450505EBD5750AEB060053
:1008A0006D100130A8422A4684BF05462A465B05E2
:1008B00037D511464046FFF74FFE00283BD0524641
:1008C00021690190FFF7FAFCA289019B22F4906252
:1008D00042F08002A281A5EB0A0203EB0A006561E7
:1008E000A260236120603546B2465946524600F068
:1008F0008FFBA068D9F808102368451B8E1B03EBFB
:100900000A00A5602060C9F808601EB3083757E9DF
:1009100002B6002EFAD0B542AA46B3D93546B24641
:10092000E3E7404600F0F0FB03460028D3D12169FD
:100930004046FFF7AFFD0C23C8F80030A389002222
:1009400043F040034FF0FF30A381C9E9012203B017
:10095000BDE8F08F0020C9F8040003B0BDE8F08FB7
:100960002DE9F04F92468A8915069DB0884681464A
:100970001C4603D50A69002A00F0EF800022099284
:100980009AF800307E4D039420228DF829203022E1
:100990008DF82A200126002B72D0544603E014F86B
:1009A000013F002B76D0252BF9D1B4EB0A0B74D183
:1009B0002278002A64D000234FF0FF32CDE90523CE
:1009C000049307938DF853301A93013404E0049A8A
:1009D00006FA03F313430493A246052214F8011BFD
:1009E000284600F0C5FA431B0028F0D1049BD80626
:1009F00044BF20228DF8532019079AF8001044BFF5
:100A00002B228DF853202A2954D1039A11680432DD
:100A1000002903927CDB07919AF801100AF1010A80
:100A20002E2959D0574C0322204600F0A1FA40B19C
:100A3000049B001B402404FA00F0034304930AF1D2
:100A4000010A1AF8011B50488DF82810062200F000
:100A50008FFA002862D04D4B002B52D003AA00928F
:100A60004B4B424604A94846AFF3008007467A1C28
:100A700006D0099B3B4409939AF80030002B8CD197
:100A8000B8F80C305B0654BF09984FF0FF301DB02A
:100A9000BDE8F08FB4EB0A0BF2D05B4652464146FC
:100AA0004846FFF77FFE0130EAD0099B22785B447D
:100AB00009937EE7A1F13002092AB1D8079B1AF801
:100AC000011F03EB830302EB4303A1F13002092A68
:100AD000F5D92E290793A5D19AF801102A2927D1F3
:100AE000039B9AF802101A6805920433002A0AF14F
:100AF00002000393B8BF4FF0FF338246B8BF05939F
:100B000090E7039B073323F0070308330393B0E711
:100B1000494243F00203079104937DE703AA009240
:100B20001B4B424604A9484600F0CAF807469EE718
:100B3000A1F130020023092A05930AF1010A3FF6C8
:100B400071AF1AF8011F03EB830302EB4303A1F11A
:100B50003002092AF5D9059364E74021FFF7FCFC30
:100B6000C8F80000C8F8100018B14022C8F81420D6
:100B700004E70C23C9F800304FF0FF3087E700BFCF
:100B8000002F0008082F00080C2F000800000000AC
:100B9000A50700082DE9F84F92461F460A698B68A1
:100BA000DDF828909A42B8BF1A46CAF8002091F89A
:100BB00043300C46064613B10132CAF800202268C1
:100BC00091065DD5DAF800300233CAF800302268A9
:100BD00012F0060F11461ED1E168CB1A002BD8BFC8
:100BE000114618DD04F1190B4FF0000805E0E56827
:100BF000DAF80030ED1A45450CDD01235A46394636
:100C00003046C847013008F10108F0D14FF0FF30FD
:100C1000BDE8F88F216894F84330003B18BF0123EA
:100C20008A060AD5E1185A1C302081F84300224474
:100C300094F8451082F84310023304F14302394618
:100C40003046C8470130E1D0236803F00603042B87
:100C50001DD0A3682269934225DD4FF000089B1A3E
:100C600098441A34002501E045451CDA0123224648
:100C700039463046C847013005F10105F4D1C5E7D2
:100C800012F0060F12D0003B18BF0123D5E7DAF8A7
:100C90000030E1682269C91AA368934221EAE17829
:100CA000DDDC0029DDDC0020BDE8F88FE168DAF842
:100CB0000030CB1A002BD8BF114693DCABE700BF46
:100CC0002DE9F0470C4684B09046227E0C990746E9
:100CD000994604F14300002A33D0A2F15803DDB253
:100CE000202D67D8202B65D8DFE813F0DE006400E4
:100CF00064006400640064006400640064006400D4
:100D00006400A3006E0064006400640064006E0070
:100D1000640064006400640021007F00C00064007F
:100D20006400AE0064007F0064006400E500236896
:100D30001A0640F104810B6862691D1D0D601B6875
:100D40001A60002382462361CDF80090434603AA2F
:100D500021463846FFF71EFF013020D02369524656
:100D600041463846C847013019D02368E068039EE1
:100D70009B0719D5831B002B16DD04F1190A0025EA
:100D800004E0E068039E831BAB420DDD0123524665
:100D900041463846C847013005F10105F1D14FF011
:100DA000FF3004B0BDE8F087B042B8BF304604B0B1
:100DB000BDE8F087012384F84220236104F1420A50
:100DC000002384F84330BFE723681A0602D45E0686
:100DD00000F1C1800D682A6804350D601546002AAF
:100DE0006BDBDFF884C10A2610E023681D0640F1A2
:100DF0009C800B681D1D0D601D68DFF86CC16F2A9B
:100E00000CBF08260A26002384F843306268A260DB
:100E1000002A7FDB236823F004032360002D5BD1CD
:100E2000002A79D18246082E65D0A0EB0A00206105
:100E30008AE70B680122186804330B6004F1420A48
:100E400084F842002261BBE70B686268181D0860E5
:100E5000D3F800A00021504600F08AF8002800F0E6
:100E60008180A0EB0A0060602061A9E7236843F05D
:100E7000200323607822DFF8F4C084F845200A6854
:100E8000151D0D601D0643D4590641D51588DE0792
:100E900044BF43F020032360002D44D1236823F096
:100EA000200323601026AEE7582384F84530DFF88E
:100EB000B8C02368E3E72368DCE76268A2602D21FD
:100EC000002AC5F1000584F8431002DB23F0040377
:100ED0002360DFF894C00A268246B5FBF6F306FBD2
:100EE00013512A461CF801100AF8011DB2421D4692
:100EF000F3D2082E99D12368D90796D56268236961
:100F00009A4292DC30230AF8013C0AF1FF3A8CE75E
:100F10001568BCE7002DDFD19CF8003084F8423022
:100F200004F1420A7FE710266DE713F0400F0B68CB
:100F300003F104050D600CBF1D681D885DE713F00B
:100F4000400F0B68626903F104050D601B6814BF54
:100F50001A801A60F5E60A68B2F9005004320A6095
:100F60002A463CE760687FE7142F0008282F000816
:100F700001F0FF01102A2BDB10F0070F08D010F84A
:100F8000013B013A8B422DD010F0070F42B3F6D14E
:100F9000F0B441EA012141EA014122F007047FF067
:100FA00000070023F0E80256083C85EA010586EABE
:100FB000010685FA47F5A3FA87F586FA47F6A5FAFA
:100FC00087F68EB9EED1F0BC01F0FF0102F0070206
:100FD00032B110F8013B013A83EA010313B1F8D1B1
:100FE0000020704701387047002D06BF3546033892
:100FF000073815F0010F07D1013015F4807F02BFCB
:10100000013015F4C03F0130F0BC0138704700BF1B
:1010100088420DD98B1883420AD900EB020CBAB171
:10102000624613F801CD02F801CD9942F9D170471B
:101030000F2A0ED8034602F1FF3C4AB10CF1010C15
:10104000013B8C4411F8012B03F8012F6145F9D1C4
:10105000704740EA01039B0750D1A2F1100370B51D
:1010600001F1200C23F00F0501F1100E00F1100426
:10107000AC441B095EF8105C44F8105C5EF80C5C34
:1010800044F80C5C5EF8085C44F8085C5EF8045CAC
:1010900044F8045C0EF1100EE64504F11004E9D1A9
:1010A000013312F00C0F01EB031102F00F0400EBFF
:1010B000031327D0043C24F003064FEA940C1E448B
:1010C0001C1F8E465EF8045B44F8045FB442F9D1FD
:1010D0000CF1010402F0030203EB840301EB840131
:1010E00002F1FF3C4AB10CF1010C013B8C4411F8B8
:1010F000012B03F8012F6145F9D170BD02F1FF3CCE
:1011000003469BE72246EBE7F8B51446F9B1CAB1AE
:1011100006460D4600F020F8A04202D32F4638467E
:10112000F8BD21463046FFF717FA07460028F6D0EB
:1011300022462946FFF7C2F830462946FFF7AAF9AA
:101140003846F8BD2746FFF7A5F93846F8BDBDE893
:10115000F8401146FFF700BA51F8040C0028A0F13E
:101160000400BCBF0B58C018704700BF53B94AB940
:10117000002908BF00281CBF4FF0FF314FF0FF309F
:1011800000F074B9ADF1080C6DE904CE00F006F87A
:10119000DDF804E0DDE9022304B070472DE9F047F3
:1011A000089D04468E46002B4DD18A42944669D94B
:1011B000B2FA82F252B101FA02F3C2F1200120FA2E
:1011C00001F10CFA02FC41EA030E94404FEA1C487C
:1011D000210CBEFBF8F61FFA8CF708FB16E341EA78
:1011E000034306FB07F199420AD91CEB030306F1FE
:1011F000FF3080F01F81994240F21C81023E63441F
:101200005B1AA4B2B3FBF8F008FB103344EA0344C2
:1012100000FB07F7A7420AD91CEB040400F1FF33D7
:1012200080F00A81A74240F207816444023840EA14
:101230000640E41B00261DB1D4400023C5E900434D
:101240003146BDE8F0878B4209D9002D00F0EF80D0
:101250000026C5E9000130463146BDE8F087B3FA03
:1012600083F6002E4AD18B4202D3824200F2F980EB
:10127000841A61EB030301209E46002DE0D0C5E9EE
:10128000004EDDE702B9FFDEB2FA82F2002A40F03A
:101290009280A1EB0C014FEA1C471FFA8CFE01263D
:1012A000200CB1FBF7F307FB131140EA01410EFBE1
:1012B00003F0884208D91CEB010103F1FF3802D288
:1012C000884200F2CB804346091AA4B2B1FBF7F082
:1012D00007FB101144EA01440EFB00FEA64508D9A5
:1012E0001CEB040400F1FF3102D2A64500F2BB80E2
:1012F0000846A4EB0E0440EA03409CE7C6F1200731
:10130000B34022FA07FC4CEA030C20FA07F401FA76
:1013100006F31C43F9404FEA1C4900FA06F3B1FBFF
:10132000F9F8200C1FFA8CFE09FB181140EA014164
:1013300008FB0EF0884202FA06F20BD91CEB010101
:1013400008F1FF3A80F08880884240F28580A8F159
:1013500002086144091AA4B2B1FBF9F009FB1011AB
:1013600044EA014100FB0EFE8E4508D91CEB010149
:1013700000F1FF346CD28E456AD90238614440EAEC
:101380000840A0FB0294A1EB0E01A142C846A6466C
:1013900056D353D05DB1B3EB080261EB0E0101FAF5
:1013A00007F722FA06F3F1401F43C5E90071002652
:1013B0003146BDE8F087C2F12003D8400CFA02FCA8
:1013C00021FA03F3914001434FEA1C471FFA8CFEB8
:1013D000B3FBF7F007FB10360B0C43EA064300FBA8
:1013E0000EF69E4204FA02F408D91CEB030300F146
:1013F000FF382FD29E422DD9023863449B1B89B2FD
:10140000B3FBF7F607FB163341EA034106FB0EF385
:101410008B4208D91CEB010106F1FF3816D28B4232
:1014200014D9023E6144C91A46EA004638E72E46FE
:10143000284605E70646E3E61846F8E64B45A9D2F6
:10144000B9EB020864EB0C0E0138A3E74646EAE765
:10145000204694E74046D1E7D0467BE7023B614413
:1014600032E7304609E76444023842E7704700BF7C
:1014700084B000220092154B196B41F004011963EE
:10148000196B01F00401009100990192196B41F070
:1014900080011963196B01F0800101910199029299
:1014A000196B41F001011963196B01F001010291FF
:1014B000029903921A6B42F002021A631B6B03F04B
:1014C00002030393039B04B0704700BF003802403F
:1014D00030B595B005464C221E4901A8FEF7EEFE38
:1014E000002409E0002214AB03EB840333F84C1C06
:1014F000194801F0C0F90134122C29DC0D2C0EDC46
:1015000045FA04F313F0010FECD0012214AB03EB06
:10151000840333F84C1C104801F0ADF9EBE745FAB1
:1015200004F313F0010F09D0012214AB03EB840381
:1015300033F84C1C094801F09EF9DCE7002214AB9B
:1015400003EB840333F84C1C044801F094F9D2E710
:1015500015B030BDD42A0008000802400004024043
:1015600070B50E4615460D4C021E18BF01224FF4F1
:101570008071204601F07FF9321E18BF01224FF41E
:101580000071204601F077F92A1E18BF01224FF49E
:101590008061204601F06FF970BD00BF000002407D
:1015A00000B587B00023019302930393049305933E
:1015B00041F6F3030193012808D00223039301A904
:1015C000054801F071F807B05DF804FB01230293B0
:1015D00002230493F3E700BF0000024030B589B056
:1015E0000020FFF7DDFF6C460E4D0FCD0FC495E8D0
:1015F0000F0084E80F000024254600E00134072C8A
:101600000DDC08AB03EB840333F8201C064801F023
:101610002BF90128F2D10123A3401D44EEE728460F
:1016200009B030BD202B00080000024070B588B022
:1016300006460120FFF7B4FF6C46134D0FCD0FC4D3
:1016400095E80F0084E80F00002409E0002208ABB1
:1016500003EB840333F8201C0C4801F00CF901342F
:10166000072C0EDC46FA04F313F0010FEED0012232
:1016700008AB03EB840333F8201C044801F0FBF8AB
:10168000EDE708B070BD00BF202B0008000002404D
:1016900038B505460C46012211461046FFF760FF9B
:1016A0002846FFF715FF2046FFF7C0FF012211462D
:1016B0000020FFF755FF002201211046FFF750FFE1
:1016C000012211460020FFF74BFF01221146104670
:1016D000FFF746FF38BD08B5AA2145F25550FFF780
:1016E000D7FF552142F6AA20FFF7D2FF802145F20D
:1016F0005550FFF7CDFFAA2145F25550FFF7C8FF1F
:10170000552142F6AA20FFF7C3FF102145F255509C
:10171000FFF7BEFF962001F065F908BD38B5044615
:101720000D46AA2145F25550FFF7B2FF552142F66A
:10173000AA20FFF7ADFFA02145F25550FFF7A8FF03
:1017400029462046FFF7A4FF38BD10B5FFF7C0FEBD
:101750000020FFF725FF012200210846FFF700FFC8
:10176000FFF73CFF0446012211461046FFF7F8FE42
:10177000204610BD38B505460C46AA2145F2555005
:10178000FFF786FF552142F6AA20FFF781FF90213F
:1017900045F25550FFF77CFF0020FFF7D6FF286089
:1017A0000120FFF7D2FF2060F02145F25550FFF7EE
:1017B0006FFF38BD30B585B00546002412E01C49E6
:1017C00001A8FEF751FF01A8FEF77AFF4FF0FF33A3
:1017D00082B201A9174800F05CFB04F00F030F2B45
:1017E00014D00134144B9C421FDC2046FFF7ADFFA0
:1017F000C2B28DF80F20002DE1D14FF0FF3301224E
:101800000DF10F010B4800F044FBEAE70B4B1B689E
:10181000ADF800301B0C8DF802304FF0FF33022280
:101820006946044800F035FBDBE705B030BD00BF7A
:10183000402B000898000020FEFF0700A82E00089B
:1018400070B58AB00024059406940794089409940E
:101850004FF6FF730593012606960225089505A904
:10186000084800F021FF009401940294039404942A
:101870001F230093019603956946034800F014FF67
:101880000AB070BD000802400004024000B587B0F5
:101890000023019302930393049305934FF4E063B1
:1018A0000193012302930223049301A9024800F04B
:1018B000FBFE07B05DF804FB0000024010B50446D3
:1018C000FEF7FEFE4FF0FF3382B22146014800F0E2
:1018D000E0FA10BD9800002010B582B00C48FFF768
:1018E000EDFF00240DE04FF0FF3301220DF1070161
:1018F000084800F034FB9DF807102046FFF70EFF64
:101900000134072CEFDD0448FFF7D8FF02B010BD0B
:10191000482B000898000020682B000872B6FEE7EC
:1019200008B50A480A4B03604FF4E13343600023D3
:101930008360C36003610C2242618361C36100F074
:1019400078FA00B908BDFFF7E9FF00BF9800002052
:101950000044004000B595B03022002108A8FEF7F1
:1019600047FD002303930493059306930793019384
:101970001F4A116C41F080511164126C02F08052C8
:101980000192019A02931B490A6822F4404242F4F0
:1019900000420A600A6802F440420292029A02215E
:1019A000089101220B9210220C920E910F9310922B
:1019B0004FF4A8731193042312930723139308A8D9
:1019C00000F036FB80B90F2303930221049100231A
:1019D00005934FF480520692079303A800F08EFD02
:1019E00020B915B05DF804FBFFF798FFFFF796FFED
:1019F000003802400070004070B584B000F0C6FFAF
:101A0000FFF7A8FFFFF734FDFFF78AFF0020FFF77D
:101A1000C7FDFFF715FFFFF739FF02A903A8FFF77E
:101A2000A9FE0D20FEF73AFC05460D20FEF736FC18
:101A300004463D4E039A31462846FEF715FE029AAB
:101A400031462046FEF710FE384E3046FFF736FF8F
:101A50003748FFF733FF3748FFF730FF3648FFF7C7
:101A60002DFF3648FFF72AFF3548FFF727FF30469E
:101A7000FFF724FF3348FFF721FF3348FFF71EFF2E
:101A80003248FFF71BFF3248FFF718FF3148FFF7D6
:101A900015FF3148FFF712FF4FF0FF3301220DF120
:101AA00006012E4800F05BFA9DF80630313B042B0E
:101AB00036D8DFE803F0030A101626002848FFF79F
:101AC000FDFE0120FFF776FED4E72648FFF7F6FE7D
:101AD000FFF701FECEE72448FFF7F0FEFFF7FCFE1C
:101AE000C8E72248FFF7EAFE2148FFF7E7FE28464D
:101AF000FFF7E4FE1F48FFF7E1FE2046FFF7DEFE9A
:101B0000B8E71D48FFF7DAFE4FF0FF3301220DF171
:101B10000701124800F023FA0020FFF74BFEFEE712
:101B20001648FFF7CBFEA5E7742B0008802B0008B2
:101B3000D82B0008002C0008582C0008B02C0008F6
:101B4000082D0008442D00088C2D0008A42D000845
:101B5000B82D0008E42D0008FC2D00089800002096
:101B6000202E0008342E0008482E00086C2E000895
:101B7000842E00089C2E0008AC2E0008D42E0008ED
:101B8000FEE7FEE7FEE7FEE7FEE7704770477047B7
:101B900008B500F015FF08BD82B0002100910B4B85
:101BA0005A6C42F480425A645A6C02F480420092A9
:101BB000009A01911A6C42F080521A641B6C03F077
:101BC00080530193019B02B0704700BF0038024070
:101BD00000B589B0002303930493059306930793FC
:101BE0000268144B9A4202D009B05DF804FB002150
:101BF000019103F5FA331A6C42F400321A641A6C3C
:101C000002F400320192019A02911A6B42F0010231
:101C10001A631B6B03F001030293029B0C230393D3
:101C2000022304930723079303A9034800F03CFD14
:101C3000DAE700BF0044004000000240026802F101
:101C40000C0353E8003F23F490730C3242E8003158
:101C50000029F3D1026802F1140353E8003F23F096
:101C60000103143242E800310029F3D1036B012B48
:101C700005D0202380F842300023036370470268B8
:101C800002F10C0353E8003F23F010030C3242E84A
:101C900000310029F3D1ECE738B504460268136936
:101CA00023F44053C1680B431361836802691343F3
:101CB00042691343C2691A430168CB6823F416438F
:101CC00023F00C031343CB600268536923F4407381
:101CD00081690B4353610368314A934206D002F590
:101CE0008062934202D000F0BFFC01E000F0CCFC27
:101CF000E369B3F5004F29D00021031849411B18AF
:101D000041F10001C90041EA5371DB001818636812
:101D10004FEA83024FEA937341F10001FFF726FA7D
:101D2000204DA5FB00325109642303FB11031B0165
:101D30003233A5FB03235B0903F0F00202EB01122F
:101D400003F00F03216813448B6038BD0023021891
:101D500043EB0301121841F10001C90041EA52713D
:101D6000D200101841F10001626892185B41FFF740
:101D7000FDF90C4DA5FB00325109642303FB11034F
:101D8000DB003233A5FB03235B095A0002F4F8722F
:101D900002EB011203F00703216813448B60D4E7C0
:101DA000001001401F85EB512DE9F04383B005463B
:101DB0000E4617469946DDF828802C68246836EAD6
:101DC00004030CBF4FF0010C4FF0000CBC4528D1B0
:101DD000B8F1FF3FF1D000F0FFFDA0EB0900404556
:101DE00023D8B8F1000F22D02B68DA6812F0040F64
:101DF000E3D0802EE1D0402EDFD01A6812F0080F19
:101E0000DBD0002401941A6801925B680193019B66
:101E10002846FFF713FF08236B6485F84040012034
:101E200000E0002003B0BDE8F0830320FAE70320C0
:101E3000F8E760B310B5044690F8413013B324239B
:101E400084F841302268D36823F40053D3602046DD
:101E5000FFF722FF2268136923F49043136122687D
:101E6000536923F02A0353612268D36843F4005373
:101E7000D36000206064202384F8413084F842302D
:101E8000606310BD80F84030FFF7A2FED7E7012065
:101E900070472DE9F04182B01E4690F84130DBB228
:101EA000202B56D104460D469046002955D00AB93C
:101EB00001204FE000234364212380F8413000F0EB
:101EC0008BFD0746A4F82480A4F82680A368B3F508
:101ED000805F02D04FF0000814E023692BB34FF06D
:101EE00000080FE0202384F84130032032E038F866
:101EF000023B2268C3F308035360E28C92B2013ABA
:101F000092B2E284E38C9BB293B100963B460022EE
:101F100080212046FFF748FF0028E3D1002DE6D0BE
:101F200015F8012B23685A60E7E7A8460025E9E782
:101F300000963B46002240212046FFF735FF18B9A6
:101F4000202384F8413005E0202384F84130032029
:101F500000E0022002B0BDE8F0810120FAE72DE99F
:101F6000F04182B01E4690F84230DBB2202B59D1AE
:101F700004460D469046002958D00AB9012052E087
:101F800000234364222280F84220036300F024FDF2
:101F90000746A4F82C80A4F82E80A368B3F5805FD0
:101FA00002D04FF000081CE0236913B14FF0000885
:101FB00017E0A846002514E0202384F842300320CF
:101FC00031E023685B68C3F3080328F8023B03E0B1
:101FD00023685B682B700135E28D92B2013A92B2B0
:101FE000E285E38D9BB2C3B100963B4600222021DF
:101FF0002046FFF7D9FE0028DED1002DE1D0A368EE
:10200000B3F5805FE4D013B92369002BE0D02368D7
:102010005B6803F07F032B70DDE7202384F84230F8
:10202000002000E0022002B0BDE8F0810120FAE7C4
:10203000002800F0E08170B582B00446036813F018
:10204000010F3BD09F4B9B6803F00C03042B2CD05B
:102050009C4B9B6803F00C03082B21D06368B3F5FD
:10206000803F4FD0B3F5A02F52D0964B1A6822F480
:1020700080321A601A6822F480221A606368002B8A
:1020800050D000F0A9FC05468E4B1B6813F4003FAE
:1020900014D100F0A1FC401B6428F5D90320B1E164
:1020A000884B5B6813F4800FD8D0864B1B6813F401
:1020B000003F03D06368002B00F09F81236813F07A
:1020C000020F54D07F4B9B6813F00C0F3ED07D4B1A
:1020D0009B6803F00C03082B33D0E368002B68D017
:1020E000794B01221A6000F077FC0546754B1B689E
:1020F00013F0020F54D100F06FFC401B0228F5D9F9
:1021000003207FE16F4A136843F480331360B5E71F
:102110006C4B1A6842F480221A601A6842F48032CA
:102120001A60ABE700F058FC0546664B1B6813F4D9
:10213000003FC3D000F050FC401B6428F5D90320B9
:1021400060E1604B5B6813F4800FC6D15D4B1B6888
:1021500013F0020F03D0E368012B40F05081594A7D
:10216000136823F0F803216943EAC103136023686D
:1021700013F0080F42D063696BB3534B0122C3F8CD
:10218000802E00F029FC05464E4B5B6F13F0020FCA
:1021900034D100F021FC401B0228F5D9032031E1A5
:1021A000484A136823F0F803216943EAC103136026
:1021B000DDE7454B00221A6000F00EFC0546414B5E
:1021C0001B6813F0020FD2D000F006FC401B02285F
:1021D000F5D9032016E13C4B0022C3F8802E00F015
:1021E000FBFB0546374B5B6F13F0020F06D000F088
:1021F000F3FB401B0228F5D9032003E1236813F009
:10220000040F77D02F4B1B6C13F0805F33D100236A
:1022100001932C4B1A6C42F080521A641B6C03F031
:1022200080530193019B0125284B1B6813F4807F89
:1022300023D0A368012B34D0052B38D0214B1A6F43
:1022400022F001021A671A6F22F004021A67A368CB
:10225000002B3DD000F0C0FB06461A4B1B6F13F05D
:10226000020F46D100F0B8FB801B41F28833984240
:10227000F3D90320C6E00025D6E7144A136843F4D7
:102280008073136000F0A8FB0646104B1B6813F424
:10229000807FCED100F0A0FB801B0228F5D903205F
:1022A000B0E0084A136F43F001031367CFE7054B13
:1022B0001A6F42F004021A671A6F42F001021A679D
:1022C000C5E700BF003802400000474200700040F0
:1022D00000F082FB0646524B1B6F13F0020F08D032
:1022E00000F07AFB801B41F288339842F3D9032037
:1022F00088E0EDB9A369002B00F08380484A92681A
:1023000002F00C02082A51D0022B17D0454B0022B4
:102310001A6600F061FB0446414B1B6813F0007F16
:1023200042D000F059FB001B0228F5D9032069E0D8
:102330003B4A136C23F080531364DBE7394B0022D4
:102340001A6600F049FB0546354B1B6813F0007F09
:1023500006D000F041FB401B0228F5D9032051E0D4
:10236000E369226A1343626A43EA8213A26A52084B
:10237000013A43EA0243E26A43EA0263284A5360AD
:10238000284B01221A6600F027FB0446244B1B68E9
:1023900013F0007F06D100F01FFB001B0228F5D9C7
:1023A00003202FE000202DE000202BE0012B2BD07C
:1023B0001B4B5B6803F48001E269914226D103F074
:1023C0003F02216A8A4223D1616A47F6C0721A40ED
:1023D000B2EB811F1ED103F44031A26A5208013AC8
:1023E000B1EB024F18D103F07063E26AB3EB026FF6
:1023F00014D1002006E001207047012002E00120F6
:1024000000E0002002B070BD0120FBE70120F9E7E9
:102410000120F7E70120F5E70120F3E70120F1E7CC
:10242000003802400000474208B5314B9B6803F07A
:102430000C03042B57D0082B57D12D4B5A6802F0B0
:102440003F025B6813F4800F2AD0294B5968C1F30F
:10245000881C4FEA4C11B1EB0C006EEB0E0E4FEAEC
:102460008E1343EA90638101091A63EB0E03DB00CC
:1024700043EA5173C90011EB0C0C43F100035902FC
:1024800000234FEA4C2041EADC51FEF76FFE184B67
:102490005B68C3F3014301335B00B0FBF3F025E05D
:1024A000134B5968C1F3881C4FEA4C11B1EB0C0077
:1024B0006EEB0E0E4FEA8E1343EA90638101091A08
:1024C00063EB0E03DB0043EA5173C90011EB0C0C04
:1024D00043F10003990200234FEA8C2041EA9C510A
:1024E000FEF744FED3E7034800E0034808BD00BF01
:1024F0000038024000127A000024F400002800F0A6
:102500009B8070B50D4604464F4B1B6803F00703D4
:102510008B4208D2CBB24C4A1370136803F0070306
:102520008B4240F08B80236813F0020F17D013F01A
:10253000040F04D0454A936843F4E0539360236842
:1025400013F0080F04D0414A936843F4604393604A
:102550003E4A936823F0F003A1680B43936023681D
:1025600013F0010F32D06368012B21D09A1E012A8B
:1025700025D9364A126812F0020F61D033498A68B1
:1025800022F0030213438B6000F026FA06462F4B1D
:102590009B6803F00C036268B3EB820F16D000F067
:1025A0001BFA801B41F288339842F0D9032042E0A5
:1025B000264A126812F4003FE0D101203BE0234A92
:1025C000126812F0007FD9D1012034E01E4B1B6845
:1025D00003F00703AB4207D9EAB21B4B1A701B6822
:1025E00003F00703AB422DD1236813F0040F06D08C
:1025F000164A936823F4E053E1680B439360236821
:1026000013F0080F07D0114A936823F4604321693F
:1026100043EAC1039360FFF707FF0C4B9B68C3F3CA
:1026200003130B4AD35CD8400A4B18600A4B186856
:1026300000F086F9002070BD012070470120FAE704
:102640000120F8E70120F6E7003C02400038024094
:10265000E82E00086C00002068000020014B18687C
:10266000704700BF6C00002008B5FFF7F7FF044B70
:102670009B68C3F38223034AD35CD84008BD00BFE4
:1026800000380240F82E000808B5FFF7E7FF044BBA
:102690009B68C3F34233034AD35CD84008BD00BFF4
:1026A00000380240F82E000800230F2B00F2D280E1
:1026B00070B582B060E085685E000324B44025EA0E
:1026C0000405CC68B4402C438460456825EA0205C3
:1026D0004C68C4F300129A402A4342605AE0DC0876
:1026E000083450F8246003F0070295000F22AA4036
:1026F00026EA020E0A69AA4042EA0E0240F82420A5
:102700005CE0042200E0002202FA0EF22A430234C6
:10271000514D45F82420514A94686FEA0C0224EA8E
:102720000C054E6816F4801F01D04CEA04054B4C92
:10273000A560E46802EA04054E6816F4001F01D0A3
:102740004CEA0405454CE560646802EA04054E68FD
:1027500016F4003F01D04CEA0405404C6560246843
:1027600022404D6815F4803F01D04CEA04023B4CF6
:10277000226001330F2B6BD801229A400C6804EAC7
:10278000020C32EA0404F4D14C6804F00304013C66
:10279000012C90D94A6802F00302032A09D0C468C8
:1027A0005D000322AA4024EA02048A68AA40224368
:1027B000C2604A6802F00302022A90D004684FEA1D
:1027C000430E032202FA0EF224EA02044A6802F0DF
:1027D000030202FA0EF2224302604A6812F4403FFA
:1027E000C7D0002201921E4A546C44F480445464C1
:1027F000526C02F480420192019A9C08A51C164A70
:1028000052F8255003F003024FEA820E0F2202FA1B
:102810000EF225EA0205134A90423FF474AF02F526
:10282000806290420ED002F5806290420CD002F598
:10283000806290420AD002F5806290423FF461AF1C
:10284000072261E701225FE702225DE703225BE7DF
:1028500002B070BD704700BF00380140003C01402D
:1028600000380240000002400369194201D00120F3
:102870007047002070470AB1816170470904816187
:1028800070470000074AD36823F4E0631B041B0C65
:10289000000200F4E060034343F0BF6343F40033FD
:1028A000D360704700ED00E000B5194BDB68C3F35F
:1028B0000223C3F1070CBCF1040F28BF4FF0040C36
:1028C00003F1040EBEF1060F18D9033B4FF0FF3E93
:1028D0000EFA0CFC21EA0C0199400EFA03F322EAED
:1028E0000303194300280BDB0901C9B200F1604062
:1028F00000F5614080F800135DF804FB0023E5E774
:1029000000F00F000901C9B2024B1954F4E700BFEF
:1029100000ED00E014ED00E00138B0F1807F0BD253
:102920004FF0E0235861054AF02182F8231000207F
:10293000986107221A6170470120704700ED00E09E
:1029400010B504460E4B18784FF47A73B3FBF0F3CE
:102950000C4A1068B0FBF3F0FFF7DEFF68B90F2CEC
:1029600001D901200AE0002221464FF0FF30FFF795
:102970009BFF054B1C60002000E0012010BD00BF44
:10298000640000206C0000206800002008B50B4B9C
:102990001A6842F400721A601A6842F480621A607F
:1029A0001A6842F480721A600320FFF76BFF002060
:1029B000FFF7C6FFFFF7F0F8002008BD003C02401B
:1029C000034A1168034B1B780B441360704700BF28
:1029D000E000002064000020014B1868704700BF31
:1029E000E000002038B50446FFF7F6FF0546B4F1D5
:1029F000FF3F02D0044B1B781C44FFF7EDFF401B48
:102A0000A042FAD338BD00BF64000020034AD2F8C8
:102A1000883043F47003C2F88830704700ED00E05E
:102A200010B503460C4A0D490D48006840B10C48EA
:102A300000680344521A934206D8094A136010BD35
:102A40000748084C0460F2E7FDF7FEFB0C23036027
:102A50004FF0FF30F3E700BF0080012000040000CA
:102A6000E4000020E8000020DFF834D0FFF7CEFFBC
:102A70000C480D490D4A002302E0D458C4500433D9
:102A8000C4188C42F9D30A4A0A4C002301E01360AF
:102A90000432A242FBD3FDF7DDFBFEF7ADFF70472A
:102AA0000080012000000020700000204C2F000852
:102AB00070000020E8000020FEE70000F8B500BF2D
:102AC000F8BC08BC9E467047F8B500BFF8BC08BC0F
:042AD0009E46704767
:102AD40001000000020000000400000008000000E3
:102AE40010000000200000004000000080000000F2
:102AF40000010000000200000004000000080000C3
:102B0400001000000020000001000000020000008E
:102B14000400000008000000100000000100000094
:102B24000200000000080000001000001000000077
:102B340020000000400000008000000025303258D2
:102B44002000000057616974696E6720666F722007
:102B540066696C6520746F20666C6173682E2E2E16
:102B64000D0A000066696E69736865640D0A0000E9
:102B7400307825303258200D0A0000003D3D3D3D9F
:102B84003D3D3D3D3D3D3D3D3D3D3D3D3D3D3D3D71
:102B94003D3D3D3D3D3D3D3D3D3D3D3D3D3D3D3D61
:102BA4003D3D3D3D3D3D3D3D3D3D3D3D3D3D3D3D51
:102BB4003D3D3D3D3D3D3D3D3D3D3D3D3D3D3D3D41
:102BC4003D3D3D3D3D3D3D3D3D3D3D3D3D3D3D3D31
:102BD4003D0D0A00205F5F5F5F5F205F5F5F5F5FA7
:102BE400205F5F5F5F5F205F5F5F5F5F205F5F5FAE
:102BF4005F5F205F5F5F5F5F0D0A00007C20202025
:102C04005F5F7C2020205F5F7C20205F20207C2071
:102C14005F5F20207C20202020207C20202020207A
:102C24007C2020205F5F5F205F5F5F205F5F5F200D
:102C34005F5F5F205F5F5F205F5F5F205F5F5F5F5D
:102C44005F205F5F5F5F5F205F5F5F205F5F5F0D9F
:102C54000A0000007C2020205F5F7C2020205F5F32
:102C64007C2020205F5F7C202020202D7C20207C65
:102C740020207C207C207C207C20207C202E207C1A
:102C840020205F7C202E207C202E207C20205F7C36
:102C9400202E277C20202020207C20202020207C07
:102CA400202D5F7C20205F7C0D0A00007C5F5F5F2D
:102CB4005F5F7C5F5F5F5F5F7C5F5F7C20207C5F2A
:102CC4005F7C5F5F7C5F5F5F5F5F7C5F7C5F7C5F7F
:102CD4007C20207C20205F7C5F7C207C5F5F5F7C8D
:102CE4005F20207C5F7C207C5F5F2C7C5F7C5F7C32
:102CF4005F7C5F7C5F7C5F7C5F5F5F7C5F7C0D0AD9
:102D040000000000202020202D204179616275738D
:102D14006120323032352020202020202020202025
:102D240020202020202020202020207C5F7C2020A8
:102D3400202020202020207C5F5F5F7C0D0A000083
:102D440048656C6C6F2077656C636F6D6520746F7C
:102D54002074686520454550524F4D2070726F674E
:102D640072616D6D657221205768617420776F758B
:102D74006C6420796F75206C696B6520746F2064B6
:102D84006F3F0D0A000000005B315D2044756D70DB
:102D940020526F6D20617320636861720D0A000018
:102DA4005B325D20457261736520636869700D0A4A
:102DB400000000005B335D2050726F6772616D200C
:102DC4006368697020766961205541525420284116
:102DD40053434949206D6F6465290D0A00000000C2
:102DE4005B345D204964656E746966792064657638
:102DF4006963650D0A0000005B355D2044756D70E4
:102E040020526F6D2061732066696C6520284153E0
:102E1400434949206D6F6465290D0A0044756D703E
:102E2400696E6720524F4D2E2E2E0D0A00000000B1
:102E340045726173696E6720436869702E2E2E0D8A
:102E44000A0000004C61756E6368696E67207072D9
:102E54006F6772616D6D696E672073657175656EFC
:102E640063652E2E2E0D0A004964656E74696679B9
:102E7400696E67206465766963652E2E2E0D0A00DF
:102E84004D616E7566616374757265722049442084
:102E94003D200D0A00000000446576696365204901
:102EA40044203D200D0A000044756D70696E672052
:102EB400524F4D2061732066696C652C20707265D9
:102EC400737320616E79206B65792E2E2E0D0A00A6
:102ED400496E76616C696420696E707574210D0A9F
:102EE40000000000000000000000000001020304D4
:102EF400060708090000000001020304232D302BFB
:102F040020000000686C4C00656667454647000079
:102F1400303132333435363738394142434445460B
:102F240000000000303132333435363738396162CD
:082F3400636465660000000003
:082F3C0060E2FF7F01000000CC
:042F44002902000856
:042F4800010200087A
:102F4C000400002000000000000000000000000051
:102F5C000000000000000000000000000000000065
:102F6C000000000000000000000000000000000055
:102F7C000000000000000000000000000000000045
:102F8C000000000000000000000000000000000035
:102F9C000000000000000000000000000000000025
:102FAC000000000001000000100000000024F400EC
:0400000508002A695C
:00000001FF
